:03800000028100FA
:06800B00438CDC05083285
:2081000075810890F001E4F0438901D2AFD2A9D28C128117021954740090F000F0E50812E9
:2081200083687B0A12835F1283B545F0700302813402811D7400F508E5906480F59090F0C3
:2081400000E00490F000F014743075F084C0E0C0F090F000E075F000C0E0C0F090F000E065
:2081600075F000C0E0C0F090F000E075F000C0E0C0F0740475F0001281837FF812834902EB
:20818000811D2223F42581F81284061281CF12840602819E78FB12833D8682088683E06011
:2081A0002D1281ADA380F778FB12833DE63099FDC299F599B40A17740D80F2E430980C30AE
:2081C00098FDC298E599B40D02740A75F00022128316868208868308E4FEFFE070061283D2
:2081E00016E4F022B42551A3E0B42D05430780A3E0B4300343074024D0B40A00500BCE75D2
:20820000F00AA42EFEA3E080EEE0B46413E60886F030F7084307201283ABA6F018F6800334
:20822000B4750543070A8021B478054307108019B46F104307088011128316F0A3128316F8
:20824000A38095B462624307027A00C004C005C006C007AB0753031F7C00E60886F0128376
:2082600071A6F018F6EDD007D006D005D0042430B43A0040022407C0E00AE645F070CC12E4
:208280008316A902EF30E505742DF0A30A12831FD0E0F0A3D9FA0808EF30E7A1EAC39E5037
:2082A0009C7420F0A30A80F4B4630DAA0112831612831FE6F0A380DEB47331C082C0838615
:2082C000820886837A00E06004A30A80F9868318868212831612831F128316E0A3128316C6
:2082E0006004F0A380F2D005D00480AAB4691B86017A00E76004090A80F912831612831FD3
:208300008601E76091F009A380F8F97A0112831612831FE9809ECDC583CDCCC582CC22EE3F
:20832000601A8FF020F715C002EAC39E500C742030F6027430F0A30A80EFD00222C82581E1
:20834000C822C92581C97A0022D083D082CF2581F581CFC082C08322CF2581F581CF227C01
:2083600000CB30E7011CCB2275F00030E70215F022C002C001AAF0F97E007D007F11C3E91F
:2083800033F9EA33FADF08F5F0E9D001D00222ED33FDEE33FEC3ED9BF5F0EE9C40E0ADF06D
:2083A000FED380DB14B4FF0215F0221283A4F4C5F0F4C5F0221283E84029801E1283E840B3
:2083C000227017801E1283E840107017800C1283E8501080051283FC6009E4F5F02212839A
:2083E000FC60F7E4F5F00422C39BC5F09C20E70720D207C345F02220D2F9D322C5F0C39C77
:208400007003E5F09B2290F001E0A360F8E0FFA3E0A3CF2582F582EF3583F58380EBFBE0A4
:20842000CB22FCE0FBA3E0CC22FAE0F9A3E0CA220A2068656C6C6F20776F726C6420257585
:0784400020257820256200D1
:00000001FF
